:020000020000FC
:1000000012C0189518951895189518955DC068C078
:1000100018951895189573C01895189518951895F2
:100020001895189518950FE50DBF04E00EBF0FEF5A
:1000300004BBACE0B1E080E29EE49BBD8ABDE0E0A1
:10004000F1E005E001930CED0193EC30D1F709B735
:10005000086109BF0AE00EBDE0E0F1E003E309B981
:1000600000E000BD06E800BD579A549A7894EC3041
:10007000F1F71A32E1F7F894112766277727AA9546
:100080000E910053602F0E9100532AE0029F600DE5
:100090000E91005324E6029F600D711D88EE93E0DF
:1000A0000E91005321F0680F791F0A95FBCFAA9596
:1000B0000E910053000FC0E0D1E0C00F7993688328
:1000C000ACE0B1E07894D3CFFFB60F9331E035BB0D
:1000D000EE27019109BD019108BD0F91FFBE189552
:1000E000FFB6330F35BB71916191EC3031F048B5FB
:1000F00059B5460F571F59BD48BDFFBE1895FFB6ED
:100100000F930CB10D930A3209F4102F0F91FFBE1B
:02011000189540
:00000001FF
